:100000000C942A010C9445010C9445010C94450173
:100010000C9445010C9445010C9445010C94450148
:100020000C9445010C9445010C9445010C94450138
:100030000C9445010C9445010C9445010C94450128
:100040000C9445010C9445010C94851B0C944501BE
:100050000C9445010C9445010C9445010C94450108
:100060000C9445010C944501756E6B6E6F776E2094
:10007000636F6D6D616E643A20006572726F7220FD
:1000800073796E63696E67206469736B0A007379B4
:100090006E63006572726F72206372656174696E5F
:1000A00067206469726563746F72793A20006D6BC2
:1000B00064697220006572726F7220777269746968
:1000C0006E6720746F2066696C650A006572726FD6
:1000D00072207365656B696E67206F6E20006572B4
:1000E000726F72206F70656E696E6720007772693B
:1000F000746520006572726F722063726561746945
:100100006E672066696C653A2000746F75636820BD
:10011000006572726F722064656C6574696E672029
:1001200066696C653A2000726D20006572726F72AC
:100130002072656164696E67206469736B20696E03
:10014000666F0A006469736B006572726F72206F6C
:1001500070656E696E67200063617420006C7300C7
:100160006469726563746F7279206E6F7420666F54
:10017000756E643A2000636420006F70656E696E6E
:100180006720726F6F74206469726563746F72792F
:10019000206661696C65640A006F70656E696E67E0
:1001A0002066696C6573797374656D206661696C2E
:1001B00065640A006F70656E696E672070617274A5
:1001C0006974696F6E206661696C65640A004D4DE3
:1001D000432F534420696E697469616C697A617454
:1001E000696F6E206661696C65640A006672656598
:1001F0003A20202000666F726D61743A2000777299
:100200002E70722E3A2000636F70793A2020200001
:1002100073697A653A20202000646174653A202071
:10022000200073657269616C3A20307800726576DF
:100230003A202020200070726F643A202020006F46
:10024000656D3A20202020006D616E75663A202091
:100250003078000011241FBECFEFD4E0DEBFCDBF49
:1002600011E0A0E0B1E0EAEAF8E302C005900D92E7
:10027000A230B107D9F713E0A2E0B1E001C01D92AE
:10028000A33CB107E1F70C94C0120C940000FC01F0
:10029000892B11F0118210820895CF93DF93FC0116
:1002A000D9018081853E29F1882319F12D913C9156
:1002B0001197ED018A819B812817390799F44C83A6
:1002C0005D836E837F8383858F3011F080E205C06C
:1002D00080818295880F807E805EFD01808780E02E
:1002E00090E009C083858F3021F02F5F3F4F2D9321
:1002F0003C9381E090E0DF91CF910895EF92FF92DF
:100300000F931F93CF93DF93EC017A018B01B90117
:100310008881853E09F4CCC0882309F4C9C0F9015D
:1003200087A190A5A1A5B2A50097A105B10521F4CB
:10033000E7A2F0A601A712A76115710509F4B8C0DC
:10034000209709F4B5C09881992309F4B1C0AE0192
:10035000455F5F4F8B858F3099F5892F99278F7374
:1003600090702DE030E0AC01429FC001439F900DA2
:10037000529F900D11249C012D5030400197809781
:1003800008F093C0FB01E20FF31F898180838B810A
:1003900081838D8182838F818383898584838E8508
:1003A0008583888986838A8987838C8980878E89DB
:1003B0008187888D82878C8D83878E8D848775C099
:1003C000FB0180818823B9F580E090E0382FFE01A1
:1003D000E80FF91F2081203249F0FB01E80FF91FD7
:1003E00020833F5F01968830910581F7FB01808172
:1003F000853011F485EE80838885803211F4832F57
:1004000016C0FB01E30FF11D8EE28083832F8F5F07
:10041000DE01232F2C5FFD019085903241F0FB011E
:10042000E80FF11D90838F5F11968217A1F7FB01F2
:10043000E80FF11D1082FA018081FB0180A38B8DF2
:100440009927982F88272A8D3327822B932B92A3C5
:1004500081A32D8D332744275527542F432F322F27
:1004600022278E8D9927AA27BB27DC019927882769
:10047000282B392B4A2B5B2B8C8D9927AA27BB273E
:10048000282B392B4A2B5B2B8F8D9927AA27BB272B
:10049000B82FAA2799278827282B392B4A2B5B2B83
:1004A00023A334A345A356A303C081E090E002C078
:1004B00080E090E0DF91CF911F910F91FF90EF903E
:1004C00008950F931F93CF93DF93CDB7DEB7229795
:1004D0000FB6F894DEBF0FBECDBFDC01892BA9F1AA
:1004E0006230710590F10D911C911197660F771F85
:1004F00088279927FD012681378140855185620F24
:10050000731F841F951FD801ED91FC9122E030E00C
:10051000AE014F5F5F4F09958823B9F08A81992713
:10052000382F222789819927282B392B211531052E
:1005300071F0BFEF273F3B0741F0C9014096079795
:1005400020F0EFEF283F3E0710F020E030E0C90137
:1005500022960FB6F894DEBF0FBECDBFDF91CF91CC
:100560001F910F9108954F925F926F927F928F9299
:100570009F92AF92BF92CF92DF92EF92FF920F9332
:100580001F93CF93DF93CDB7DEB722970FB6F894C2
:10059000DEBF0FBECDBF5C01009709F44BC06230D7
:1005A000710508F447C0FC016680778080849184DF
:1005B0002E010894411C511C660F771F6B01EE241D
:1005C000FF24C60CD71CE81CF91CD501ED91FC9149
:1005D0000190F081E02D22E030E0A201C701B601D8
:1005E0000995882339F18A819927182F0027898155
:1005F0009927082B192B01151105F9F0C801409610
:100600000897C0F0BFEF083F1B0710F000E010E0B4
:1006100019821A82D501ED91FC910480F581E02DBB
:1006200022E030E0A201C701B6010995B801012B13
:1006300021F0C2CF80E090E002C081E090E02296FD
:100640000FB6F894DEBF0FBECDBFDF91CF911F91E3
:100650000F91FF90EF90DF90CF90BF90AF909F9061
:100660008F907F906F905F904F9008952F923F9260
:100670004F925F926F927F928F929F92AF92BF92B2
:10068000CF92DF92EF92FF920F931F93CF93DF935E
:10069000CDB7DEB72C970FB6F894DEBF0FBECDBF37
:1006A0003C012B011A01009709F495C0DC01ED9182
:1006B000FC91208131813C872B870480F581E02DDE
:1006C000FA87E987FC0186819781A085B1858D83B2
:1006D0009E83AF83B88782859385A485B585B695BB
:1006E000A795979587959C838B836A01AA24BB2441
:1006F0008824992444C0C401880F991F7C010027D5
:1007000011272D813E814F815885E20EF31E041F73
:10071000151F22E030E0AE014F5F5F4FC801B70107
:10072000AB85BC85FD010995882309F454C08981F6
:10073000882311F58A818823F9F4C214D30419F4AB
:100740008FEF898303C0A9828B2D99278A8322E0AA
:1007500030E0AE014F5F5F4FC801B701E985FA8510
:100760000995882391F00894C108D108C114D104D7
:1007700011F454010CC054010894811C911C2B816C
:100780003C818216930609F0B6CFCD2801F532E000
:100790004316510410F1A9828B2D99278A83440CAA
:1007A000551CB201882799272D813E814F8158859C
:1007B000620F731F841F951F22E030E0AE014F5F70
:1007C0005F4FA985BA85FD010995882331F4B501EC
:1007D000C3010E94B302AA24BB24C5012C960FB604
:1007E000F894DEBF0FBECDBFDF91CF911F910F9167
:1007F000FF90EF90DF90CF90BF90AF909F908F9041
:100800007F906F905F904F903F902F900895CF9280
:10081000DF92EF92FF920F931F93CF93DF93CDB7A9
:10082000DEB760970FB6F894DEBF0FBECDBF7C0178
:100830006230710518F480E090E027C0FC01C088A8
:10084000D1880081118162507040882799279601D4
:10085000442755270E94EC1B9B01AC01F7016689D8
:100860007789808D918D620F731F841F951FF8010A
:10087000A681B781EE24FF2405EF16E09601AE01B4
:100880004F5F5F4FFD010995992760960FB6F89469
:10089000DEBF0FBECDBFDF91CF911F910F91FF90B3
:1008A000EF90DF90CF900895FC01892B11F0118219
:1008B000108208952F923F924F925F926F927F9293
:1008C0008F929F92AF92BF92CF92DF92EF92FF9260
:1008D0000F931F93CF93DF93CDB7DEB72C970FB64F
:1008E000F894DEBF0FBECDBF3C0178876F835A8777
:1008F0004987009709F4FCC0672B09F4F9C0452B20
:1009000009F4F6C0FC01A5A4B6A4C7A4D0A825A1EB
:1009100036A147A150A569857A85CB01AA27BB27B7
:100920008A0D9B1DAC1DBD1D281739074A075B07A3
:1009300038F42A193B093A872987232B09F4DBC0AD
:10094000D3018D919C91FC01808991899A8389833F
:10095000F30101A8F2A9E02DFC87EB87BC018827F1
:1009600099276B837C838D839E83EF2BE1F5F301C5
:1009700003A0F4A1E02DFC87EB87EF2B39F4A11441
:10098000B104C104D10409F4B6C0B2C0A114B104C9
:10099000C104D10441F1860175012B803C804D805A
:1009A0005E805094409430942094211C311C411C52
:1009B000511C10C06B857C85D3018D919C910E9448
:1009C00061029C878B87892B09F492C0E20CF31C8F
:1009D000041D151D6B817C818D819E81E616F706B5
:1009E0000807190738F7C601B5012B813C814D81F5
:1009F0005E810E94321C2B0189849A84D3018D91DF
:100A00009C91A980BA80A418B5088A149B0408F4A4
:100A10005401FC01C080D180720100271127868912
:100A20009789A08DB18DE80EF91E0A1F1B1F2B851B
:100A30003C8522503040B901882799272E5F3F4FCF
:100A40003C872B872B813C814D815E810E94EC1B72
:100A5000E60EF71E081F191FD601CD90DC909501F8
:100A60004F815885C801B701F6010995882339F1EE
:100A70008A189B08C501AA27BB27F30125A536A51F
:100A800047A550A9280F391F4A1F5B1F25A736A766
:100A900047A750ABC501840D951D29813A81821766
:100AA0009307A0F06B857C85808191810E94610213
:100AB0009C878B87892B41F4F30112AA11AA4985DF
:100AC0005A854819590919C0442455242B853C8559
:100AD000F30132AB21AB8114910439F06F81788539
:100AE0006A0D7B1D78876F8389CF49855A8505C03C
:100AF0004FEF5FEF02C040E050E0CA012C960FB606
:100B0000F894DEBF0FBECDBFDF91CF911F910F9143
:100B1000FF90EF90DF90CF90BF90AF909F908F901D
:100B20007F906F905F904F903F902F900895FC01C1
:100B3000892B11F0118210820895FC01892B19F480
:100B400080E090E0089516A615A681E090E0089553
:100B50008F929F92AF92BF92CF92DF92EF92FF92CD
:100B60000F931F93CF93DF93CDB7DEB72C970FB6BC
:100B7000F894DEBF0FBECDBF6C015B01892B09F479
:100B800052C06115710509F44EC0FB01E7A0F0A445
:100B900001A512A5E114F1040105110509F443C0F2
:100BA0004E010894811C911CD601ED91FC9101909D
:100BB000F081E02D2CE030E0A401C801B7010995D7
:100BC000882389F185EE8983D601ED91FC9104801B
:100BD000F581E02D2CE030E0A401C801B7010995B2
:100BE000882309F18C858F3049F480E290E0A0E001
:100BF000B0E0E80EF91E0A1F1B1FD6CFF50161A158
:100C000072A16115710519F481E090E00AC0C60176
:100C10000E94B30220E030E0882311F021E030E0B0
:100C2000C901992702C080E090E02C960FB6F89495
:100C3000DEBF0FBECDBFDF91CF911F910F91FF900F
:100C4000EF90DF90CF90BF90AF909F908F900895DE
:100C500008950895FC01892B29F460E070E080E09C
:100C600090E008956285738584859585969587952E
:100C70007795679562507040804090402089318917
:100C8000442755270E94EC1B08952F923F924F92C4
:100C90005F926F927F928F929F92AF92BF92CF920C
:100CA000DF92EF92FF920F931F93CF93DF93CDB715
:100CB000DEB7A5970FB6F894DEBF0FBECDBF1C01FF
:100CC000892B09F456C01A82198280E28B83F101C4
:100CD000468057806084718482849384A484B58420
:100CE00037C0FEEF8F16FFEF9F06F0E0AF06F0E093
:100CF000BF0628F02EEF3FEF3DA32CA302C09DA21C
:100D00008CA2D101ED91FC910280F381E02D6E0166
:100D10000894C11CD11CB6EDEB2EB6E0FB2E0CA145
:100D20001DA120E230E0AE014C5F5F4FC301B20174
:100D300009958823F1F00CA11DA1C801AA27BB27A2
:100D4000480E591E6A1E7B1E881A990AAA0ABB0AF7
:100D500081149104A104B10421F6F1016089718923
:100D60008827992729813A81442755270E94EC1B1F
:100D700004C060E070E080E090E0A5960FB6F894C3
:100D8000DEBF0FBECDBFDF91CF911F910F91FF90BE
:100D9000EF90DF90CF90BF90AF909F908F907F901B
:100DA0006F905F904F903F902F900895AC01D901C4
:100DB000F9016281FC0112C081819927982F88274F
:100DC00020813327822B932B892B39F48D919C9191
:100DD0001197019611969C938E9332968E2F841BB9
:100DE000861750F381E090E0089520E1FC01119214
:100DF0002A95E9F780E190E008952F923F924F9273
:100E00005F926F927F928F929F92AF92BF92CF929A
:100E1000DF92EF92FF920F931F93CF93DF93CDB7A3
:100E2000DEB7E5970FB6F894DEBF0FBECDBF1C014D
:100E30007DA76CA7009709F4F7C0672B09F4F4C0ED
:100E4000FC0163A074A025A536A53FA72EA740806E
:100E500051806114710409F050C04114510409F427
:100E6000E0C0D201ED91FC91A280B3809E012F5F82
:100E70003F4F89E0F90111928A95E9F78EA59FA568
:100E80009C838B83F20162897389848995890689A1
:100E90001789061B170BFAE08F2E912C8C0E9D1EC6
:100EA0006901EDE4EE2EE1E0FE2E20E230E0A40147
:100EB000F5010995882309F4B4C04D805E806F80E8
:100EC0007884411451046104710409F4AAC08BE2CE
:100ED000ACA5BDA51D928A95E9F709851127CCA47B
:100EE000DDA47EE7E72E71E0F72E20E230E0A401DA
:100EF000C301B201F501099584C04114510409F4FC
:100F000090C0FC0182A184FF8CC0F2010088F189AD
:100F1000E02DFBA7EAA7CF01AA27BB2788AB99AB97
:100F2000AAABBBABDE011196BDABACABEEEFFFEFF6
:100F30006E0E7F1EB3018827992722E030E0620EF3
:100F4000731E28A939A94AA95BA90E94EC1BF201CA
:100F500086889788A08CB18C860E971EA81EB91E15
:100F600089E0ACA9BDA91D928A95E9F7EEA5FFA578
:100F7000FC83EB83D201ED91FC91AE01465F5F4FA4
:100F80000280F381E02D6E010894C11CD11C6DE438
:100F9000E62E61E0F62E0AA51BA520E230E0C50191
:100FA000B40109958823E9F18D809E80AF80B884D3
:100FB00081149104A104B10441F4B301C2010E945F
:100FC00061023C01892B69F1B1CF8BE2ECA5FDA553
:100FD00011928A95E9F7D201ED91FC9109851127CB
:100FE0000280F381E02DCCA4DDA43EE7E32E31E0C6
:100FF000F32E20E230E0AE01465F5F4FC501B40141
:101000000995882371F0ECA5FDA58081882349F01E
:10101000F10185A596A5019696A785A781E090E0A8
:1010200005C0F10116A615A680E090E0E5960FB682
:10103000F894DEBF0FBECDBFDF91CF911F910F910E
:10104000FF90EF90DF90CF90BF90AF909F908F90E8
:101050007F906F905F904F903F902F9008952F92C8
:101060003F924F925F926F927F928F929F92AF9238
:10107000BF92CF92DF92EF92FF920F931F93CF9385
:10108000DF93CDB7DEB7AC970FB6F894DEBF0FBED7
:10109000CDBF6C01009709F4A2C1FC018481958148
:1010A000892B09F49CC186819781892B09F497C10A
:1010B00002E011E01CA70BA78091020190910301AF
:1010C000892B09F08CC18AE1D8011D928A95E9F734
:1010D000D0920301C09202010185128523853485D7
:1010E00089E0000F111F221F331F8A95D1F70AA331
:1010F0001BA32CA33DA3C901B801655F7F4F8F4F90
:101100009F4F0190F081E02D29E130E0AE014F5F6B
:101110005F4F0995882309F45EC129813A80FB81DC
:10112000F8A74C813D815E812F8048845984AA8430
:101130008D859927F82FEE278C859927E82BF92B99
:10114000EE888F89688D798D309709F444C199278D
:10115000AA27BB276624782E892E9A2E862F9927B8
:10116000AA27BB27DC0199278827682A792A8A2A97
:101170009B2A8E2D9927AA27BB27682A792A8A2A93
:101180009B2A872F9927AA27BB27B82FAA279927F9
:101190008827682A792A8A2A9B2A61147104810483
:1011A000910479F48A2D9927782F6627852D992720
:1011B000682B792B6115710509F40DC13B01882459
:1011C0009924832D9927982F88279FA38EA3822F58
:1011D00099270EA11FA1082B192B1FA30EA3842D45
:1011E0009927982F88279AA789A7822D992769A5DB
:1011F0007AA5682B792B7AA769A7832F9927982F2F
:101200008827242F3327822B932B8C0122273327E7
:101210000A8F1B8F2C8F3D8FBF0188279927252F81
:101220003327442755270E94EC1B6E8F7F8F88A39E
:1012300099A3840173012A8D3B8D4C8D5D8DE21A3B
:10124000F30A040B150BE61AF70A080B190B8EA10B
:101250009FA1019729A53AA545E0220F331F4A9582
:10126000E1F7820F931F6EA17FA10E940B1C8827BC
:101270009927E61AF70A080B190B68A5262F3327BA
:1012800044275527C801B7010E94321C19012A01C1
:10129000DA01C901855F9F40A040B0408050904F67
:1012A000A040B04008F097C086E0F60180870BA50B
:1012B0001CA50E5F1F4F88E1D8011D928A95E9F7A2
:1012C000025010401CA70BA7EEA1FFA15F01CC2488
:1012D000DD24C401B301A60195010E94EC1B6093BB
:1012E0000401709305018093060190930701C601E4
:1012F000B5012A8D3B8D4C8D5D8D0E94EC1B7B01D1
:101300008C012AA13BA14CA15DA1E20EF31E041F9A
:10131000151FE0920801F092090100930A01109351
:101320000B01220C331C441C551C44E050E060E0CF
:1013300070E0240E351E461E571E20920C0130927E
:101340000D0140920E0150920F016EA17FA170938A
:1013500011016093100178A5872F9927AEA1BFA135
:10136000FC01AE9FC001AF9F900DBE9F900D112458
:1013700090931301809312016E8D7F8D88A199A1A6
:10138000A60195010E94EC1B6E0D7F1D801F911F11
:1013900060931401709315018093160190931701C7
:1013A00009A51AA5980144275527A5E0220F331F48
:1013B000441F551FAA95D1F7620F731F841F951FF5
:1013C000609318017093190180931A0190931B0187
:1013D0008BA59CA506C0109203011092020180E02B
:1013E00090E0AC960FB6F894DEBF0FBECDBFDF9194
:1013F000CF911F910F91FF90EF90DF90CF90BF9012
:10140000AF909F908F907F906F905F904F903F90A4
:101410002F9008952F923F924F925F926F927F92FA
:101420008F929F92AF92BF92CF92DF92EF92FF92F4
:101430000F931F93CF93DF93CDB7DEB723970FB6EC
:10144000F894DEBF0FBECDBF1C019B01892B09F4B0
:10145000C2C04115510509F4BEC0FA010190002037
:10146000E9F7E41BF50BCF010B966DE070E00E94ED
:101470000B1C6F5F6B83F90143A054A0411451040E
:1014800051F0662477244301AA24BB246501EE248D
:10149000FF2487010BC0F101A288B388C488D588D6
:1014A000E688F788008D118D350146011A82AE1449
:1014B000BF04C006D10609F05EC04114510409F40E
:1014C0008AC0A114B104C104D10479F1B201C101EF
:1014D0000E946102009741F541E050E0B201C10174
:1014E0000E9436038C01892B09F475C0025010400C
:1014F000B801882799270E5F1F4FF1012089318994
:10150000442755270E94EC1B3B014C01F1018689C1
:101510009789A08DB18D680E791E8A1E9B1EB80119
:10152000C1010E9407045AC02C01F101E088F18832
:10153000002711272EEF3FEF420E531EB2018827DE
:101540009927A2E0B0E04A0E5B1EA80197010E9415
:10155000EC1B5B016C01F10186899789A08DB18D2F
:10156000A80EB91ECA1EDB1EEA0CFB1C0C1D1D1D9D
:10157000350146011A82D101ED91FC910190F08173
:10158000E02D21E030E0AE014F5F5F4FC601B501B5
:101590000995882301F18981853E11F0882379F42A
:1015A000BA81BF5FBA83EB81BE17C0F480E290E0DE
:1015B000A0E0B0E0A80EB91ECA1EDB1E78CF90E2F4
:1015C000692E712C812C912C6A0C7B1C8C1C9D1C0F
:1015D000640153016BCF662477244301C401B30136
:1015E00023960FB6F894DEBF0FBECDBFDF91CF912B
:1015F0001F910F91FF90EF90DF90CF90BF90AF9031
:101600009F908F907F906F905F904F903F902F9022
:1016100008954F925F927F928F929F92AF92BF9266
:10162000CF92DF92EF92FF920F931F93CF93DF93AE
:10163000CDB7DEB7A0970FB6F894DEBF0FBECDBF13
:10164000FC018B01892B09F41AC16115710509F49C
:1016500016C10190F081E02D44805580FB01A7A0C8
:10166000B0A4C1A4D2A401900020E9F73197FE2EC6
:10167000F61A8F2D99270C966DE070E00E941F1CC2
:10168000762E4BE050E060E270E0CE0101960E94C1
:10169000A71B6EE270E0C8010E94E11BFC010097ED
:1016A000C1F0DC0111968181882399F0FD01019040
:1016B0000020E9F73197EA1BFB0BFE1AFA944E2F34
:1016C000E43008F043E05527BD01CE0109960E94A1
:1016D0009E1BCE010196F8E0FF1588F04F2D55278F
:1016E000B8010E949E1BD8018C918E3219F5F80129
:1016F00081818E3209F482818823D9F01BC0DC01FC
:10170000F80188E001900D928150E1F7F80181A184
:10171000982F92959F70803A10F4905D01C09F5968
:101720008F708A3010F4805D01C08F599F83888745
:1017300001C077248981853E11F485E089837CE0AE
:10174000872E912C8C0E9D1E85E1D4011D928A95C9
:10175000E9F7F80180A18C8781A192A18B8F892F55
:1017600099278C8F83A194A1A5A1B6A18D8F292F34
:101770003A2F4B2F55272E8F9D01442755272F8F0A
:101780008B2F9927AA27BB2788A3672D7727882720
:10179000992725E0660F771F881F991F2A95D1F793
:1017A0006A0D7B1D8C1D9D1D20E230E0AE014F5F58
:1017B0005F4FF2010995882309F461C0E980FE01B9
:1017C000329694018E2D8695E794EE24E794E82ACC
:1017D0008191E80EE217F307A9F7F72C4E01089460
:1017E000811C911C0D50104044C040E250E06FEF4E
:1017F00070E0C4010E94A71B8DE0F89ED001112467
:10180000A00FB11F91E0F401E90FF11D8C918083CD
:10181000892F8F5FF401E80FF11D10829E5F9B30CE
:1018200021F09A3119F49CE101C09EE08C9188234B
:1018300021F09F3110F41196E6CFF982F71419F4D4
:101840008F2D806489838FE08C87EE861D861B8EAA
:101850001C8E20E230E0A401C601B501F201099519
:1018600080E290E0A0E0B0E0A80EB91ECA1EDB1E28
:10187000FA94FF2009F0B9CF81E090E002C080E047
:1018800090E0A0960FB6F894DEBF0FBECDBFDF91FB
:10189000CF911F910F91FF90EF90DF90CF90BF906D
:1018A000AF909F908F907F905F904F9008952F9270
:1018B0003F924F925F926F927F928F929F92AF92E0
:1018C000BF92CF92DF92EF92FF920F931F93CF932D
:1018D000DF93CDB7DEB72E970FB6F894DEBF0FBEFD
:1018E000CDBF6C011A012B01009709F4E2C0FC0185
:1018F000E3A0F4A00190F081E02D80899189E114AA
:10190000F10431F4411551056105710509F4BDC0BB
:10191000420131019C01442755272F83388749878D
:101920005A8750954095309521953F4F4F4F5F4FC7
:101930002B873C874D875E8711C0B701D6018D91FB
:101940009C910E9461020097B9F02B853C854D85E2
:101950005E85620E731E841E951E7C018F819885A4
:10196000A985BA858B839C83AD83BE838615970535
:10197000A805B90510F3A0C05701C401B3012B811C
:101980003C814D815E810E94321C8901B90188270A
:1019900099272B813C814D815E810E94EC1B66154D
:1019A00077058805990510F40F5F1F4FA801B7014F
:1019B000D6018D919C910E943603009709F479C05D
:1019C000EF2821F4F60194A383A35C01F60125A27C
:1019D00036A247A250A6211431044104510411F447
:1019E00014A213A2B6016E5F7F4FD6018D919C9118
:1019F0000E94090B882309F45CC0211431044104BE
:101A0000510429F4B501F601808191813CC02B81FC
:101A10003C814D815E812615370548055905A8F1A1
:101A2000D6010D911C910115110579F1B2E0AB16AB
:101A3000B10458F1B501C8010E9461027C018FEF29
:101A400089838A83F80180809180AA0CBB1CB50130
:101A5000882799272681378140855185620F731F1A
:101A6000841F951FF401A481B58122E030E0AE010E
:101A70004F5F5F4FFD010995882339F0E114F104B0
:101A800021F0B701C8010E94B302F60185A596A511
:101A9000A7A5B0A9281639064A065B0638F4F60150
:101AA00025A636A647A650AA12AA11AA81E090E060
:101AB00009C080E090E006C05701E114F10409F488
:101AC0005CCF84CF2E960FB6F894DEBF0FBECDBF8D
:101AD000DF91CF911F910F91FF90EF90DF90CF900A
:101AE000BF90AF909F908F907F906F905F904F903E
:101AF0003F902F900895CF92DF92EF92FF920F9335
:101B00001F93CF93DF93EC016B01892B09F446C03F
:101B10006115710509F442C08DA59EA5AFA5B8A9B0
:101B2000413059F0413018F04230C1F50CC0FB0192
:101B3000E080F1800281138113C0FB01E080F1801D
:101B40000281138109C0FB01E080F18002811381D1
:101B50008DA19EA1AFA1B8A5E80EF91E0A1F1B1FFB
:101B60008DA19EA1AFA1B8A58E159F05A007B107B5
:101B700038F4B801A701CE010E94570C882371F0F8
:101B8000EDA6FEA60FA718AB1AAA19AAF601E082C5
:101B9000F1820283138381E090E002C080E090E054
:101BA000DF91CF911F910F91FF90EF90DF90CF9039
:101BB00008952F923F924F925F926F927F928F92F1
:101BC0009F92AF92BF92CF92DF92EF92FF920F93CC
:101BD0001F93CF93DF93CDB7DEB72A970FB6F89454
:101BE000DEBF0FBECDBF5C011B0158874F8300973E
:101BF00009F43BC1672B09F438C1452B09F435C101
:101C0000FC0165A476A487A490A885A196A1A7A1AC
:101C1000B0A586159705A805B90508F426C1208149
:101C20003181F9010088F189E02DFA83E983F5011A
:101C300001A8F2A9E02DFA87E98789819A81AA276C
:101C4000BB278B839C83AD83BE83EF2B09F059C0E8
:101C5000F50103A0F4A1E02DFA87E987EF2BA9F4A1
:101C6000611471048104910409F0FFC041E050E067
:101C700060E070E0C9010E9436039A878987F50108
:101C800094A383A3892B09F4F0C0F501E5A4F6A47D
:101C900007A510A9E114F1040105110549F531C0AA
:101CA0008B819C81AD81BE81E81AF90A0A0B1B0B5E
:101CB00069857A85D5018D919C910E94610200977A
:101CC00019F09A87898714C0E114F1040105110500
:101CD00009F0CBC041E050E069857A85F50180814B
:101CE00091810E943603009709F4BFC09A878987C3
:101CF0008B819C81AD81BE81E816F9060A071B071E
:101D000078F6C401B3012B813C814D815E810E9434
:101D1000321C2B016F807884D5018D919C91898034
:101D20009A80841895086814790408F44301FC012A
:101D3000C080D18072010027112786899789A08DE4
:101D4000B18DE80EF91E0A1F1B1F29853A85225006
:101D50003040B901882799272E5F3F4F3A8729875E
:101D60002B813C814D815E810E94EC1BE60EF71EAB
:101D7000081F191FF601A481B5819401A101C801B2
:101D8000B701FD010995882309F446C06818790850
:101D9000C401AA27BB27F50125A536A547A550A94B
:101DA000280F391F4A1F5B1F25A736A747A750AB2F
:101DB000C401840D951D29813A818217930708F18A
:101DC00069857A85808191810E946102009719F06E
:101DD0009A87898714C06114710459F041E050E07A
:101DE00069857A85D5018D919C910E943603009773
:101DF00021F4F50112AA11AA0FC09A8789874424F9
:101E0000552429853A85F50132AB21AB6114710463
:101E100019F0280C391C80CFF50185A596A5A7A53A
:101E2000B0A9E5A0F6A007A110A5E816F9060A07D3
:101E30001B07B0F485A396A3A7A3B0A7B5016E5F57
:101E40007F4F808191810E94090B882349F4F5011D
:101E500065A476A46E187F08E5A6F6A607A710ABC2
:101E60008F8198858619970902C08FEF9FEF2A9678
:101E70000FB6F894DEBF0FBECDBFDF91CF911F919B
:101E80000F91FF90EF90DF90CF90BF90AF909F9019
:101E90008F907F906F905F904F903F902F9008951C
:101EA000CF93DF939C01FB01892B21F1672B11F16B
:101EB00080A184FF1FC080914F0190915001892B18
:101EC00019F4AFE4B1E008C080917E0190917F01E8
:101ED000892B81F4AEE7B1E0ED0122968BE201900F
:101EE00009928150E1F711963C932E93FD0116A6BD
:101EF00015A602C0A0E0B0E0CD01DF91CF9108951A
:101F0000CF93DF939C01FB01892B49F1611571058A
:101F100031F180A184FD23C080911C0190911D01AD
:101F2000892BE9F4CEE1D1E0DB018BE20D9009923F
:101F30008150E1F730931D0120931C01109249015B
:101F400010924A0110924B0110924C0181A192A172
:101F500090934E0180934D018CE191E002C080E0AE
:101F600090E0DF91CF910895CF92DF92EF92FF92B0
:101F70000F931F93CF93DF937C018B01EA01892B91
:101F800009F443C06115710509F43FC0FB0180816C
:101F90008823D9F1452BC9F1BE01C7010E94FD0676
:101FA000882351F0BE01C8010E94BA1B892BA1F7FA
:101FB000F70116A615A629C0F701C080D1808BE2D3
:101FC000FE0111928A95E9F74FE150E0B801CE0188
:101FD0000E94D21BAE01B701C6010E940A0A6FA37C
:101FE00078A789A79AA7611571058105910569F000
:101FF000BE01C6010E94090B90E0882309F491E01C
:1020000081E09827892F992702C080E090E0DF9136
:10201000CF911F910F91FF90EF90DF90CF90089597
:102020006F927F928F929F92AF92BF92CF92DF92E8
:10203000EF92FF920F931F93CF93DF933C018B019D
:102040007A01892B09F461C06115710509F45DC03D
:10205000FB018081882309F458C0452B09F455C041
:102060008F3211F40F5F1F4F8BE2F70111928A95A7
:10207000E9F780E1F70180A3F8018081882309F462
:1020800047C0B701C3010E94500F5C01892BE9F1E1
:102090006FE270E0C8010E94AE1B6C01892B41F415
:1020A000F80101900020E9F76F010894C108D108F8
:1020B0008C2D801B882E992421C0E70109900020D7
:1020C000E9F72197CE19DF09C815D905B9F4AE0192
:1020D000B701C8010E94C41B892B81F4F50111824C
:1020E0001082C00FD11F8881882391F0F70180A151
:1020F00084FF0BC086010F5F1F4FC3CFB701C5011F
:102100000E94FD068823C9F606C080E090E007C063
:1021100081E090E004C0F50111821082B2CFDF911E
:10212000CF911F910F91FF90EF90DF90CF90BF90D4
:10213000AF909F908F907F906F9008959F92AF92F5
:10214000BF92CF92DF92EF92FF920F931F93CF93A4
:10215000DF936C015B01EA01892B09F495C06115DD
:10216000710509F491C0FB018081882309F48CC0BA
:10217000452B09F489C0BE01C6010E94FD068823D3
:1021800051F0BE01C5010E94BA1B892BA1F7F601CF
:1021900016A615A679C0F601E080F18041E050E076
:1021A00060E070E0C7010E9436038C01009709F4DB
:1021B0006BC0BC01C7010E9407048BE2FE011192B3
:1021C0008A95E9F780E188A302501040B80188277A
:1021D00099270E5F1F4FF701208931894427552722
:1021E0000E94EC1BF70126893789408D518D260FFF
:1021F000371F481F591F2FA338A749A75AA7BEE268
:102200009B2E98821AA309A3BE01C7010E94090B45
:102210008823B1F18FA198A5A9A5BAA58096A11D83
:10222000B11D8FA398A7A9A7BAA79982F60183A188
:1022300094A19AA389A3BE01C7010E94090B882318
:10224000F9F04FE150E0B501CE010E94D21B1AA374
:1022500009A3AE01B601C7010E940A0A6FA378A7BD
:1022600089A79AA7611571058105910549F0BE01FD
:10227000C7010E94090B882319F081E090E006C095
:10228000B801C7010E94B30280E090E0DF91CF91D6
:102290001F910F91FF90EF90DF90CF90BF90AF9084
:1022A0009F900895EF92FF920F931F93FC01DB0123
:1022B000B80187ED97E09183808381E08C93FA01E8
:1022C0008083F9011082FB011082F70110821F91B7
:1022D0000F91FF90EF9008950F931F93CF93DF938B
:1022E000CDB7DEB769970FB6F894DEBF0FBECDBF8E
:1022F0008C01892B09F49CC0CE0101960E945419CF
:10230000882309F495C088E492E00E94611B8981CA
:102310000E94771A8AE00E94681A8FE392E00E9476
:10232000611BCE0102960E94541B8AE00E94681A2B
:1023300086E392E00E94611BCE0105960E94541B29
:102340008AE00E94681A8DE292E00E94611B8B85F0
:102350000E94771A8AE00E94681A82E292E00E9444
:10236000611B6C857D858E859F850E94A01A8AE001
:102370000E94681A89E192E00E94611B898999276D
:102380000E94B31A8FE20E94681A888999270E94D6
:10239000B31A8AE00E94681A80E192E00E94611BF1
:1023A0006A897B898C899D890E94F31A8AE00E9440
:1023B000681A87E092E00E94611B8E8999270E942B
:1023C000B31A8AE00E94681A8EEF91E00E94611BA6
:1023D000888D99270E94B31A8FE20E94681A8F890C
:1023E00099270E94B31A8AE00E94681A85EF91E04B
:1023F0000E94611B898D99270E94B31A8AE00E946E
:10240000681A8CEE91E00E94611BC8010E9445068B
:102410000E94F31A8FE20E94681AC8010E942A06DD
:102420000E94F31A8AE00E94681A81E090E002C0DC
:1024300080E090E069960FB6F894DEBF0FBECDBF86
:10244000DF91CF911F910F910895EF92FF920F931B
:102450001F93CF93DF938B017A01E9010CC0B70181
:10246000CE010E94BA1B892B31F4C8010E949D0540
:1024700081E090E008C0BE01C8010E94FD068823EB
:1024800071F780E090E0DF91CF911F910F91FF9065
:10249000EF900895EF92FF920F931F93CF93DF93E6
:1024A000CDB7DEB7AB970FB6F894DEBF0FBECDBF8A
:1024B0008C017E010894E11CF11C97010E942512F9
:1024C000882319F480E090E004C0B701C8010E949D
:1024D000800FAB960FB6F894DEBF0FBECDBFDF9175
:1024E000CF911F910F91FF90EF900895AF92BF92FF
:1024F000DF92EF92FF920F931F93CF93DF937C01B4
:10250000062F1127A80160E070E00E94A71BDD24C0
:1025100058010894A108B10823C00E946F1B182F0E
:10252000883011F08F3789F4DD20D1F0DA94F7018B
:10253000ED0DF11D108288E00E94681A80E20E9471
:10254000681A88E00E94681A0BC00E94681AF70196
:10255000EC0FFD1F1A3011F4108207C01083D394C2
:10256000CD2DDD27CA15DB05C4F2CE01DF91CF9159
:102570001F910F91FF90EF90DF90BF90AF90089563
:10258000C3E8D4E0DEBFCDBF83B7817F83BF0E94A5
:102590005C1A0E94DF18882319F48EEC91E026C2A1
:1025A00000E02FE038E14DE057E169E678E18CE3A7
:1025B00096E10E940615009781F40FEF2FE038E1B5
:1025C0004DE057E169E678E18CE396E10E9406155B
:1025D000009719F484EB91E009C20E942F084C0186
:1025E000009719F489E991E001C28E010B5D1F4F3C
:1025F000A80160E071E00E941010B801C4010E94BF
:10260000500F3C01892B19F48AE791E0EFC1C40116
:102610000E946C112DE0222E312C2C0E3D1ECE017D
:10262000805B9F4FED969FAF8EAFED978EE30E943C
:10263000681A80E20E94681A68E1C1010E9476125D
:102640008823A1F343E050E066E771E0C1010E94F6
:10265000901B892B01F58889882341F39E01205B1B
:102660003F4FAE01405F5F4FB301C4010E9425128E
:10267000882371F0BE01605B7F4FC4010E94500F40
:102680008C01892B29F0C3010E9497053801CECF18
:1026900080E691E0C9C06DE571E0C1010E94861B32
:1026A000892BE9F533C0ED96AEADBFADED970D903A
:1026B0000020E9F78D0101501040ED96EEADFFAD21
:1026C000ED970E1B1F0BCE01805B9F4F0E94541B8A
:1026D000E1968FADE19784FF02C08FE201C080E2F6
:1026E00094E2F92EF01A01C080E20E94681AFA946E
:1026F000FFEFFF16C9F7E7966CAD7DAD8EAD9FADD0
:10270000E7970E94F31A8AE00E94681ABE01605B94
:102710007F4FC3010E94FD06882329F687CF44E03E
:1027200050E068E571E0C1010E94901B892B09F01F
:1027300047C08989882309F479CFAE014F5E5F4F86
:10274000B301C4010E944A125C01892B49F0CC24D8
:10275000DD24760185E0482E512C4C0E5D1E25C0EF
:1027600089E491E00E94611BCE01419639C1C70105
:10277000B6010E94A01A8AE30E94681A820180E2D0
:102780000E94681AD8018D918D010E94771A021556
:102790001305A9F78AE00E94681A88E090E0A0E09B
:1027A000B0E0C80ED91EEA1EFB1E48E050E0B201A0
:1027B000C5010E945A0418161906CCF2C501BCC006
:1027C00064E471E0C1010E94861B892B49F4C401B5
:1027D0000E946C11882309F029CF8BE291E0F8C0A8
:1027E00043E050E067E271E0C1010E94901B892B39
:1027F00001F58889882309F419CF9E01205B3F4F9A
:10280000AE01405F5F4FB301C4010E9425128823CF
:1028100049F0BE01605B7F4FC4010E94A805882378
:1028200009F004CF81E191E00E94611BCE01409646
:10283000D7C046E050E06AE071E0C1010E94901B01
:10284000892B99F48B89882309F4F0CEAE01405B83
:102850005F4FBE016D5E7F4FC3010E94B40F88239E
:1028600009F0E4CE84EF90E0A0C046E050E06DEEC9
:1028700070E0C1010E94901B892B09F07BC08B89FD
:10288000882309F4D3CE8E010D5E1F4F02C00F5F67
:102890001F4FD8018C91803219F08823C1F7C6CE22
:1028A000F8011082AE014D5E5F4FB301C4010E947A
:1028B0004A127C01892B19F48EED90E076C020E05D
:1028C00030E040E050E017C0CA01B9012AE030E032
:1028D00040E050E00E94EC1B9B01AC018D2D99273C
:1028E00087FD9095C097AA2797FDA095BA2F280F2E
:1028F000391F4A1F5B1FF801D1800F5F1F4F8D2DBD
:1029000080538A3008F329833A834B835C8340E009
:10291000BE016F5F7F4FC7010E947B0D882379F452
:102920008CEC90E00E94611BCE0143960E94541BE8
:102930008AE00E94681AC7010E94540477CE8CE393
:102940000E94681A80E20E94681A68E1C1010E9430
:102950007612882381F3082F1127A801B101C7013E
:102960000E94D90D8017910751F385EB90E00E94EA
:10297000611BE1CF46E050E06EEA70E0C1010E94C9
:10298000901B892BB9F48B89882309F44FCEAE01B3
:10299000405B5F4FBE016D5E7F4FC3010E949E1082
:1029A000882309F043CE83E990E00E94611BCE01A9
:1029B000439616C06EE870E0C1010E94861B892B09
:1029C00051F40E94F117882309F030CE8AE790E095
:1029D0000E94611B2BCE88E690E00E94611BC10122
:1029E0000E94541B8AE00E94681A20CE0E94611B3C
:1029F00081E090E00C94541CFC01892B19F480E0D8
:102A000090E00895108681E090E008958F929F9263
:102A1000AF92BF92CF92DF92EF92FF920F93CF933C
:102A2000DF93CDB7DEB760970FB6F894DEBF0FBE69
:102A3000CDBF7C016B015A014901892B09F4AAC061
:102A4000672B09F4A7C004300CF0A4C007FD1DC01B
:102A5000602F772767FD7095E4E0660F771FEA9592
:102A6000E1F762547E4F882777FD8095982F20E10B
:102A700030E0AE014F5F5F4FF7010995882309F4FD
:102A800089C08D81882309F485C08091B501882390
:102A900009F080C0EDEAF1E081E1DF011D928A9545
:102AA000E9F7F092AE01E092AD01D092B001C09290
:102AB000AF01B092B201A092B1019092B4018092A4
:102AC000B30107FD62C08D818093B5012A8533274C
:102AD00044275527542F432F322F22278B859927A0
:102AE000AA27BB27DC0199278827282B392B4A2BBB
:102AF0005B2B89859927AA27BB27282B392B4A2BA3
:102B00005B2B8C859927AA27BB27B82FAA27992743
:102B10008827282B392B4A2B5B2B2093B601309327
:102B2000B7014093B8015093B9012E85332744274C
:102B30005527542F432F322F22278F859927AA27D5
:102B4000BB27DC0199278827282B392B4A2B5B2BA5
:102B50008D859927AA27BB27282B392B4A2B5B2B3E
:102B600088899927AA27BB27B82FAA2799278827BA
:102B7000282B392B4A2B5B2B2093BA013093BB01B6
:102B80004093BC015093BD0103C08FEF8093B5010A
:102B9000CF0102C080E090E060960FB6F894DEBFEF
:102BA0000FBECDBFDF91CF910F91FF90EF90DF90DF
:102BB000CF90BF90AF909F908F90089586B18295EF
:102BC0008F7099278095909581709070089586B147
:102BD00082958695877099278095909581709070E1
:102BE00008958EBD0DB407FEFDCF8DB58F778DBDD9
:102BF00008958FEF8EBD0DB407FEFDCF8DB58F7795
:102C00008DBD8EB599270895DF92EF92FF920F93B5
:102C10001F93D82E7A018B010E94F9158D2D8064A7
:102C20000E94F115812F9927AA27BB270E94F11531
:102C3000C801AA27BB270E94F115BB27A12F902FFF
:102C40008F2D0E94F1158E2D0E94F115DD2011F4BB
:102C500085E901C08FEF0E94F11510E00E94F9157F
:102C60008F3F19F41F5F1A30C9F799271F910F91F1
:102C7000FF90EF90DF9008952F923F924F925F92D6
:102C80006F927F928F929F92AF92BF92CF92DF927C
:102C9000EF92FF920F931F93CF93DF93CDB7DEB7E1
:102CA00024970FB6F894DEBF0FBECDBF2B013C01B9
:102CB0005A8349833C832B8390C0812C5EEF952EF1
:102CC0005FEFA52E5FEFB52E84209520A620B720BC
:102CD0004FEFC42E41E0D42EC420D520212C32E069
:102CE000332E2C183D088B819C818215930508F4A6
:102CF0001C01E090BE03F090BF030091C00310914F
:102D0000C1038E149F04A006B10609F449C0809146
:102D1000C203882351F420E032E04EEB51E0C801B9
:102D2000B7010E940D17882349F02A98B501A40124
:102D300081E10E940416882321F02A9A80E090E025
:102D400053C00E94F9158E3FE1F70EEB11E00E948F
:102D5000F915F80181938F01F3E00E3B1F07B9F7D6
:102D60008092BE039092BF03A092C003B092C103B1
:102D70008EEB91E0C80ED91EA101B60189819A811E
:102D80000E949E1BE981FA81E20DF31DFA83E9831B
:102D90000E94F9150E94F9152A9A0E94F91510C08F
:102DA0008EEB91E0C80ED91EA101B60189819A81EE
:102DB0000E949E1BE981FA81E20DF31DFA83E983EB
:102DC0008B819C81821993099C838B83C101AA27E3
:102DD000BB27480E591E6A1E7B1EEB81FC81EF2B20
:102DE00009F06BCF81E090E024960FB6F894DEBF37
:102DF0000FBECDBFDF91CF911F910F91FF90EF904C
:102E0000DF90CF90BF90AF909F908F907F906F900A
:102E10005F904F903F902F9008952F923F924F9246
:102E20005F926F927F928F929F92AF92BF92CF925A
:102E3000DF92EF92FF920F931F93CF93DF93CDB763
:102E4000DEB724970FB6F894DEBF0FBECDBF2B01BF
:102E50003C015A834983190186B182958695877012
:102E600080FF9CC0A0C0A12C7EEFB72E7FEFC72EA5
:102E70007FEFD72EA420B520C620D720C2019170A5
:102E80009C838B83812C62E0962E881A990A2814E1
:102E9000390408F44101E090BE03F090BF030091B3
:102EA000C0031091C103AE14BF04C006D10659F18E
:102EB0008091C203882359F420E032E04EEB51E0C8
:102EC000C801B7010E940D17882309F46CC0EB817B
:102ED000FC81EF2B29F4F0E08F16F2E09F0658F406
:102EE00020E032E04EEB51E0C601B5010E943C16F5
:102EF000882309F458C0A092BE03B092BF03C092C9
:102F0000C003D092C10389819A81E1E08E3B9E0784
:102F100071F0A401BC018B819C8182549E4F0E9460
:102F20009E1B1092C2032814390409F43FC02A984A
:102F3000B601A50188E10E940416882311F02A9A9F
:102F400032C08EEF0E94F1150EEB11E0F801819175
:102F50008F010E94F115F3E00E3B1F07B9F78FEFC9
:102F60000E94F1158FEF0E94F1150E94F9158F3F15
:102F7000E1F789819A81880D991D9A8389830E943E
:102F8000F9152A9A28183908C401AA27BB27480E20
:102F9000591E6A1E7B1E81E08093C20321143104F6
:102FA00009F061CF03C080E090E002C081E090E0D2
:102FB00024960FB6F894DEBF0FBECDBFDF91CF9140
:102FC0001F910F91FF90EF90DF90CF90BF90AF9047
:102FD0009F908F907F906F905F904F903F902F9039
:102FE00008958091C203882319F081E090E008954C
:102FF0006091BE037091BF038091C0039091C103A3
:1030000020E032E04EEB51E00E940D1790E0882363
:1030100009F491E081E09827892F992708954F922C
:103020005F926F927F928F929F92AF92BF92CF9258
:10303000DF92EF92FF920F931F93CF93DF935B0189
:103040006C014A01E90138012701452B61F1012B8F
:1030500051F1FF24232B11F5FF24F3941FC092019B
:10306000B601A501C401F30109958C010097F1F0A7
:10307000FF2019F4C817D907B0F09801A401C601C0
:10308000B5010E940D17882371F0C801AA27BB273C
:10309000A80EB91ECA1EDB1EC01BD10BFF20F9F6FD
:1030A0002097E9F603C080E090E002C081E090E064
:1030B000DF91CF911F910F91FF90EF90DF90CF9014
:1030C000BF90AF909F908F907F906F905F904F9048
:1030D00008952F923F924F925F926F927F928F92BC
:1030E0009F92AF92BF92CF92DF92EF92FF920F9397
:1030F0001F93CF93DF93CDB7DEB724970FB6F89425
:10310000DEBF0FBECDBF4B015C013A013C832B8378
:103110002701DA82C982452BA1F12115310589F1F8
:103120000217130770F1EF2861F11901309421940F
:1031300031083394021B130B6901EE24FF242B8109
:103140003C81A301C501B4010E943C168823C9F04B
:1031500029813A81B501A401C301F20109958823AF
:1031600099F0020D131D8B819C81800F911F2B8183
:103170003C818217930740F08C0C9D1CAE1CBF1C39
:10318000DECF80E090E002C081E090E024960FB6B0
:10319000F894DEBF0FBECDBFDF91CF911F910F918D
:1031A000FF90EF90DF90CF90BF90AF909F908F9067
:1031B0007F906F905F904F903F902F9008951F9356
:1031C000CF93DF933C983D98239A259A229A24988E
:1031D0002A9A83E58CBD8DB58E7F8DBD86B1829593
:1031E0008F7080FD17C010E00E94F9151F5F1A3024
:1031F000D9F72A98C0E0D0E040E050E060E070E00D
:1032000080E00E940416813051F081E0CF3FD80762
:1032100021F42A9A80E090E043C02196EDCFC0E0EF
:10322000D0E040E050E060E070E081E00E940416F1
:1032300080FF06C08FE7CF3FD80759F32196F1CF23
:1032400040E052E060E070E080E10E9404168823D4
:1032500001F72A9A8CB58C7F8CBD8DB581608DBDB0
:103260008FEF9FEFAFEFBFEF8093BE039093BF034D
:10327000A093C003B093C10311E01093C20320E0F8
:1032800032E04EEB51E060E070E080E090E00E94C0
:103290003C1690E0882309F491E09127892F992723
:1032A000DF91CF911F910895CF92DF92EF92FF921D
:1032B0000F931F93CF93DF93EC01892B09F4F1C097
:1032C00086B182958F7080FDECC089E1FE0111927C
:1032D0008A95E9F72A9840E050E060E070E08AE0E3
:1032E0000E940416882309F061C00E94F9158E3FE0
:1032F000E1F78E0120E6E22EF12C0E94F915282F2D
:10330000802F8C1B883028F4833090F4882359F068
:103310000CC08D3018F4893080F40DC08D3029F147
:103320008E3079F526C028832CC0F801208329C06F
:10333000F801218326C02A8724C033274427552734
:103340000E2C04C0220F331F441F551F0A94D2F7BE
:103350008B859C85AD85BE85822B932BA42BB52BAD
:103360008B879C87AD87BE870CC02295207F2F87D7
:1033700008C0922F92959F708F85892B8F872F7011
:10338000288B0F5F1F4F88EF9FEFE80EF91E90ED1F
:10339000E9169FEFF90609F0B0CF40E050E060E099
:1033A00070E089E00E940416882311F02A9A79C0FF
:1033B0000E94F9158E3FE1F7CC24DD24EE24FF2492
:1033C00000E010E00E94F915083021F1093040F4C6
:1033D000063091F00730B0F4053009F058C008C04D
:1033E0000A3041F10A3008F10E3009F050C03AC0FD
:1033F0009FE0C92EC8224BC0992783709070F82E89
:10340000EE2445C09927E82AF92AEE0CFF1CEE0CA1
:10341000FF1C3DC082958695869583709927E82A82
:10342000F92A0894E11CF11C32C0F3E0DF2ED82207
:10343000DD0C2DC0881F8827881FD82A97014427B4
:1034400055278C2D992702968D0D911D04C0220FB2
:10345000331F441F551F8A95D2F7298B3A8B4B8B0C
:103460005C8B15C0282F332726FF02C081E08D8B8F
:1034700025FF02C081E08E8B24FF02C081E08F8B8C
:103480002C7030703595279535952795288F0F5FCF
:103490001F4F0231110509F095CF2A9A81E090E083
:1034A00002C080E090E0DF91CF911F910F91FF90DB
:1034B000EF90DF90CF9008951092C50087E680933B
:1034C000C40086E08093C20088E98093C10008951B
:1034D0001F93182F8A3019F48DE00E94681A80918A
:1034E000C00085FFFCCF1093C6001F9108951F9365
:1034F000182F82958F708A3010F4805D01C0895A30
:103500000E94681A812F99278F709070212F2F7039
:103510000A971CF4822F805D02C0822F895A0E9474
:10352000681A1F9108950F931F938C01812F99277B
:103530000E94771A802F0E94771A1F910F91089589
:10354000EF92FF920F931F937B018C01C801AA2772
:10355000BB270E94931AC7010E94931A1F910F91D3
:10356000FF90EF900895DF92EF92FF920F931F93D9
:10357000CF93DF93EC0100E117E220E0EE24FF247B
:10358000CE01B8010E940B1CD62E662329F42223FB
:1035900019F40130110529F48D2D805D0E94681AFF
:1035A00021E0C8016AE070E00E940B1C0894E11C55
:1035B000F11C45E0E416F10471F08D2D9927AC0162
:1035C000409FC001419F900D509F900D1124C81B3A
:1035D000D90B8B01D5CFDF91CF911F910F91FF9028
:1035E000EF90DF9008954F925F926F927F928F924B
:1035F0009F92AF92BF92CF92DF92EF92FF920F9382
:103600001F93CF93DF937B018C01A12C2AECB22E68
:103610002AE9C22E2BE3D22E4424C0E0D0E0C80118
:10362000B701A60195010E94321C522E222341F4BB
:10363000442031F481E0A816B104C104D10431F46E
:10364000852D805D0E94681A44244394C601B5010B
:103650002AE030E040E050E00E94321C39014A018B
:103660002196CA30D10579F0652D772788279927CB
:10367000A60195010E94EC1BE61AF70A080B190B2C
:1036800064015301CCCFDF91CF911F910F91FF9037
:10369000EF90DF90CF90BF90AF909F908F907F90F2
:1036A0006F905F904F900895CF93DF93EC0103C02C
:1036B00021960E94681A88818823D1F7DF91CF91E3
:1036C0000895CF93DF93EC01FE0121968491882326
:1036D00019F00E94681AF8CFDF91CF9108959FB733
:1036E000789407C083B7816083BF889583B78E7F46
:1036F00083BF8091C00087FFF5CF9FBF8091C60038
:103700008D3009F48AE0992708951895FB01DC01B2
:103710008D910590801911F40020D1F7990B08952F
:10372000FB01DC014150504030F08D910590801933
:1037300019F40020B9F7881B990B0895FB01DC01EF
:1037400002C001900D9241505040D8F70895DC011D
:1037500001C06D9341505040E0F70895FC01019085
:10376000061629F00020D9F7882799270895319760
:10377000CF010895FB01DC018D910190801911F4B6
:103780000020D1F7990B0895FB01DC014150504016
:1037900030F08D910190801919F40020B9F7881B41
:1037A000990B0895FB01DC014150504048F0019015
:1037B0000D920020C9F701C01D9241505040E0F722
:1037C0000895FC0181E090E00190061609F4CF0114
:1037D0000020D1F701970895629FD001739FF001F7
:1037E000829FE00DF11D649FE00DF11D929FF00D91
:1037F000839FF00D749FF00D659FF00D9927729FC8
:10380000B00DE11DF91F639FB00DE11DF91FBD0152
:10381000CF0111240895AA1BBB1B51E107C0AA1FA9
:10382000BB1FA617B70710F0A61BB70B881F991F61
:103830005A95A9F780959095BC01CD01089597FB05
:10384000092E07260AD077FD04D0E5DF06D0002038
:103850001AF4709561957F4F0895F6F790958195CC
:103860009F4F0895A1E21A2EAA1BBB1BFD010DC09C
:10387000AA1FBB1FEE1FFF1FA217B307E407F50720
:1038800020F0A21BB30BE40BF50B661F771F881FFC
:10389000991F1A9469F760957095809590959B0192
:0A38A000AC01BD01CF010895FFCF78
:0238AA002F00ED
:00000001FF
